:020000040000FA
:02000000A02836
:08000800A000030EA100831209
:100010008B1C3D288B1028181A28A81C3D28B519C0
:1000200016286430010203183C281A2864300102A3
:10003000031C3C280000000000000000000000003D
:1000400000000000000000000000000000000000B0
:10005000000000002810A814A210031006180314B2
:10006000A40DA30DA20DA90B3D2828152408A70057
:100070002308A6002208A500A81081010B11210E5B
:080080008300A00E200E090010
:10014000203084008001840A80300402031CA2282D
:100150003830840086228000B30A840A7830040292
:10016000031CAA284030B1003830B0007830AF000E
:100170001230A9008316FE308505333086058312C0
:100180008501860107309F00C830831681008312E5
:10019000313090007E309200A63083169800831292
:1001A000803098000C30831699008312003083163B
:1001B0008C00831290308B0081018E018F010B1116
:1001C0008B100B108C130C138C120C120C118C1046
:1001D0000C108B171121281932218E1FEA288F014C
:1001E0008E018E160E166D220510B60BEA280A3007
:1001F000B6002721063031020318EA28AA30B200DF
:100200005D22AA30B2005D22AA30B2005D226430C5
:10021000B2005D223508B2005D226D30B2005D2271
:10022000EA286400281808000B1D08000B11A8100C
:1002300028141230A900061C22292A14831601133F
:10024000831208002A108316011783120800003950
:10025000851C0838051E0438851D0238051D013827
:10026000B500080028110608803A860005148E01A2
:100270008F010C102A1C412925090339A500A60964
:10028000A709B519CA292608B3003310B3102518D9
:100290003314A518B3149022AB009422AC000130A3
:1002A000271E5529AB070318AC0A0230271D5B290E
:1002B000AB070318AC0A3C3027050C3C0319702926
:1002C0003C302705303C031970293C3027053C3C65
:1002D000031970293C302705003C031970298B292C
:1002E000C0302705003C03197B29C0302705C03CDE
:1002F00003197B298B2903302705003C0319862924
:1003000003302705033C031986298B292C08FF3C61
:10031000031D8E298B294530B2005D2201302C024D
:10032000031DA2292C302B02031C9C292C30AB026C
:100330003330B2005D22B5293830AB073230B2001D
:100340005D22B529C8302B02031CAC29C830AB0292
:100350003230B2005D22B52964302B02031CB5296E
:100360006430AB023130B2005D222B08B3007C2236
:10037000B2005D228122B2005D224730A71BB2008D
:100380005230A71FB2005D222A30A718B200A7186A
:100390005D22502AE4302702F0300319A7004C30C8
:1003A00027020C300319A7006C3027023C300319D8
:1003B000A700EC302702FC300319A700B330270256
:1003C000F3300319A7001B3027020F300319A700D1
:1003D0003B3027023F300319A700BB302702FF3014
:1003E0000319A700443027065439031908001030B8
:1003F00027065439031908002608B3003310B31038
:1004000025183314A518B3148C22AB000A2A4530E2
:10041000B2005D22C8302B02031C142AC830AB0284
:100420003230B2005D221D2A64302B02031C1D2ACB
:100430006430AB023130B2005D222B08B3007C2265
:10044000B2005D228122B2005D222D30B2005D2219
:100450002A30B20003302606033903195D223130F9
:10046000B20050302706543903195D223230B200F1
:1004700004302706543903195D223330B20014309A
:100480002706543903195D223430B2005430270650
:10049000543903195D222A30B20027185D22502AF0
:1004A0002708B2005D222608B2005D222508B200AE
:1004B0005D22FF30B2005D2208004830310203188F
:1004C0000617031808002F08840032088000B10ABC
:1004D000AF0A3830AF1BAF0008000C1E0800B1088F
:1004E000031908003008840000089900B103B00A1D
:1004F0003830B01BB0000800B31304308A00330852
:100500008200B31704308A0033088200B317331314
:1005100007308A003308820003308A0033088200E3
:1005200005308A003308820006308A0033088200D2
:100600005034513402340134E5347134E734E63483
:1006100036346134383437341B3481341D341C345F
:10062000C1345934C934C534C3347934CB34C734B4
:10063000C2346934CA34C634C4348934CC34C8347E
:100640001234553414341334F7347534F934F8341F
:10065000483465344A3449342D3485342F342E34AB
:1006600009345D340B340A34EE347D34F034EF3425
:100670003F346D344134403424348D3426342534B1
:100680009134BF34B134A13499347334B934A934BA
:1006900095346334B534A5349D348334BD34AD34DE
:1006A00093345B34B334A3349B34C034BB34AB34A5
:1006B00097346B34B734A7349F348B345334AF340E
:1006C00092345734B234A2349A347734BA34AA34D8
:1006D00096346734B634A6349E348734BE34AE3490
:1006E00094345F34B434A4349C347F34BC34AC349C
:1006F00098346F34B834A834A0348F347B34B03499
:100700000634523408340734EB347234ED34EC34AC
:100710003C3462343E343D34213482342334223438
:10072000D9345A34E134DD34DB347A34E334DF3421
:10073000DA346A34E234DE34DC348A34E434E034EB
:10074000183456341A341934FD347634FF34FE34F8
:100750004E34663400344F343334863435343434D4
:100760000F345E3411341034F4347E34F634F534FE
:1007700045346E34473446342A348E342C342B348A
:100780000334543405340434E8347434EA34E9343A
:10079000393464343B343A341E34843420341F34C6
:1007A000CD345C34D534D134CF347C34D734D334E5
:1007B000CE346C34D634D234D0348C34D834D434AF
:1007C0001534583417341634FA347834FC34FB3486
:1007D0004B3468344D344C34303488343234313412
:1007E0000C3460340E340D34F1348034F334F2348C
:1007F0004234703444344334273490342934283418
:1008000030343034303430343034303430343034C8
:1008100030343034313431343134313431343134B2
:10082000313431343134313432343234323432349C
:100830003234323432343234323432343334333486
:100840003334333433343334333433343334333470
:100850003434343434343434343434343434343458
:100860003434343435343534353435343534353442
:10087000353435343534353436343634363436342C
:100880003634363436343634363436343734373416
:100890003734373437343734373437343734373400
:1008A00038343834383438343834383438343834E8
:1008B00038343834393439343934393439343934D2
:1008C00039343934393439343034303430343034E4
:1008D00030343034303430343034303431343134F6
:1008E00031343134313431343134313431343134E0
:1008F00032343234323432343234323432343234C8
:1009000030343134323433343434353436343734AB
:100910003834393430343134323433343434353497
:100920003634373438343934303431343234333483
:10093000343435343634373438343934303431346F
:10094000323433343434353436343734383439345B
:10095000303431343234333434343534363437345B
:100960003834393430343134323433343434353447
:100970003634373438343934303431343234333433
:10098000343435343634373438343934303431341F
:10099000323433343434353436343734383439340B
:1009A000303431343234333434343534363437340B
:1009B00038343934303431343234333434343534F7
:1009C00036343734383439343034313432343334E3
:1009D00034343534363437343834393430343134CF
:1009E00032343334343435343634373438343934BB
:1009F00030343134323433343434353436343734BB
:100A00003D34003405340134003400340034003403
:100A1000D5340034DD34D9346934003471346D3464
:100A20000034003400340034003400340034003426
:100A30000034003400340034003400340034003416
:100A4000453400344D34493400340034003400342B
:100A50001D34003425342134B1340034B934B53474
:100A60002134003429342534003400340034003477
:100A7000F93400340134FD348D340034953491342C
:100A800000340034003400340034003400340034C6
:100A900000340034003400340034003400340034B6
:100AA00000340034003400340034003400340034A6
:100AB0000034003400340034003400340034003496
:100AC0000034003400340034003400340034003486
:100AD0000034003400340034003400340034003476
:100AE0000034003400340034003400340034003466
:100AF0000034003400340034003400340034003456
:100B0000153400341D3419340034003400340034FA
:100B1000ED340034F534F1348134003489348534D3
:100B20000034003400340034003400340034003425
:100B30000034003400340034003400340034003415
:100B40005D340034653461340034003400340034E2
:100B5000353400343D343934C9340034D134CD34E3
:100B60003934003441343D3400340034003400342E
:100B70001134003419341534A5340034AD34A9349B
:100B80000934003411340D3400340034003400349E
:100B9000E1340034E934E534753400347D3479349B
:100BA00000340034003400340034003400340034A5
:100BB0000034003400340034003400340034003495
:100BC0005134003459345534003400340034003486
:100BD0002934003431342D34BD340034C534C134AB
:100BE0002D340034353431340034003400340034D2
:100BF000053400340D34093499340034A1349D3463
:100C00000134FF3400340034FF34FF34FF34FF3448
:100C10000034FF34003400340034FF340034003436
:100C2000FF34FF34FF34FF34FF34FF34FF34FF342C
:100C3000FF34FF34FF34FF34FF34FF34FF34FF341C
:100C40000034FF3400340034FF34FF34FF34FF3409
:100C50000134FF34013401340034FF3400340034F3
:100C60000034FF3400340034FF34FF34FF34FF34E9
:100C70000034FF34013400340034FF3400340034D5
:100C8000FF34FF34FF34FF34FF34FF34FF34FF34CC
:100C9000FF34FF34FF34FF34FF34FF34FF34FF34BC
:100CA000FF34FF34FF34FF34FF34FF34FF34FF34AC
:100CB000FF34FF34FF34FF34FF34FF34FF34FF349C
:100CC000FF34FF34FF34FF34FF34FF34FF34FF348C
:100CD000FF34FF34FF34FF34FF34FF34FF34FF347C
:100CE000FF34FF34FF34FF34FF34FF34FF34FF346C
:100CF000FF34FF34FF34FF34FF34FF34FF34FF345C
:100D00000034FF3400340034FF34FF34FF34FF3448
:100D10000034FF34003400340034FF340034003435
:100D2000FF34FF34FF34FF34FF34FF34FF34FF342B
:100D3000FF34FF34FF34FF34FF34FF34FF34FF341B
:100D40000034FF3400340034FF34FF34FF34FF3408
:100D50000134FF34013401340034FF3400340034F2
:100D60000034FF3400340034FF34FF34FF34FF34E8
:100D70000134FF34013401340034FF3400340034D2
:100D80000034FF3400340034FF34FF34FF34FF34C8
:100D90000034FF34003400340034FF3400340034B5
:100DA000FF34FF34FF34FF34FF34FF34FF34FF34AB
:100DB000FF34FF34FF34FF34FF34FF34FF34FF349B
:100DC0000034FF3400340034FF34FF34FF34FF3488
:100DD0000134FF34013401340034FF340034003472
:100DE0000034FF3400340034FF34FF34FF34FF3468
:100DF0000134FF34013401340034FF340034003452
:100F00000D347734773477342E346434693467346D
:100F10006934743461346C342D346234613468342F
:100F20006E342E34643465340D3453346E346F347F
:100F30006F34703479342034563430342E343634AF
:100F4000343420344D346F3474342034203420341D
:100F500020342034203420342034203420342034F1
:100F600020342034203420342034203420340D34F4
:100F7000303438342E3432343034303438340D3464
:084000000A00000006000400A4
:02400E00543D1F
:00000001FF
